:100000000C94E2020C940A030C940A030C940A0365
:100010000C940A030C94DC200C940A030C940A033D
:100020000C940A030C940A030C940A030C940A031C
:100030000C940A030C940A030C940A030C940A030C
:100040000C94731F0C940A030C940A030C940A0377
:100050000C940A030C940A030C940A030C940A03EC
:100060000C94BD1F0C940A0300000000003E5B4F7F
:100070005B3E3E6B4F6B3E1C3E7C3E1C183C7E3C08
:10008000181C577D571C1C5E7F5E1C00183C180016
:10009000FFE7C3E7FF0018241800FFE7DBE7FF30A6
:1000A000483A060E2629792926407F050507407F14
:1000B00005253F5A3CE73C5A7F3E1C1C08081C1C87
:1000C0003E7F14227F22145F5F005F5F06097F017D
:1000D0007F006689956A606060606094A2FFA29468
:1000E00008047E040810207E201008082A1C080836
:1000F0001C2A08081E101010100C1E0C1E0C303884
:100100003E3830060E3E0E06000000000000005F84
:1001100000000007000700147F147F14242A7F2AA0
:100120001223130864623649562050000807030062
:10013000001C2241000041221C002A1C7F1C2A08AE
:10014000083E080800807030000808080808000011
:1001500060600020100804023E5149453E00427F85
:10016000400072494949462141494D331814127FD4
:100170001027454545393C4A494931412111090774
:100180003649494936464949291E000014000000F5
:1001900040340000000814224114141414140041C7
:1001A00022140802015909063E415D594E7C121184
:1001B000127C7F494949363E414141227F414141BC
:1001C0003E7F494949417F090909013E4141517337
:1001D0007F0808087F00417F41002040413F017FA8
:1001E000081422417F404040407F021C027F7F0470
:1001F00008107F3E4141413E7F090909063E4151B9
:10020000215E7F09192946264949493203017F01A8
:10021000033F4040403F1F2040201F3F4038403FA9
:10022000631408146303047804036159494D4300BF
:100230007F4141410204081020004141417F0402F6
:10024000010204404040404000030708002054548D
:1002500078407F284444383844444428384444286B
:100260007F385454541800087E090218A4A49C78BE
:100270007F0804047800447D40002040403D007F1A
:100280001028440000417F40007C047804787C08FA
:100290000404783844444438FC18242418182424CE
:1002A00018FC7C08040408485454542404043F44B3
:1002B000243C4040207C1C2040201C3C4030403CE2
:1002C00044281028444C9090907C4464544C440042
:1002D00008364100000077000000413608000201A6
:1002E0000204023C2623263C1EA1A161123A404092
:1002F000207A38545455592155557941225454780F
:1003000042215554784020545579400C1E527212A7
:100310003955555559395454545939555454580030
:1003200000457C410002457D420001457C407D1234
:1003300011127DF0282528F07C5455450020545496
:100340007C547C0A097F4932494949323A44444441
:100350003A324A4848303A4141217A3A424020787C
:10036000009DA0A07D3D4242423D3D4040403D3C7D
:1003700024FF2424487E4943662B2FFC2F2BFF09A2
:1003800029F620C0887E0903205454794100004496
:100390007D413048484A32384040227A007A0A0A81
:1003A000727D0D19317D2629292F282629292926F4
:1003B00030484D4020380808080808080808382F39
:1003C00010C8ACBA2F102834FA00007B00000814C3
:1003D0002A142222142A14085500550055AA55AA99
:1003E00055AAFF55FF55FF000000FF00101010FF39
:1003F00000141414FF001010FF00FF1010F010F094
:10040000141414FC001414F700FF0000FF00FF1484
:1004100014F404FC141417101F10101F101F1414D0
:10042000141F00101010F0000000001F101010101A
:100430001F10101010F010000000FF10101010100E
:1004400010101010FF10000000FF140000FF00FF4C
:1004500000001F10170000FC04F4141417101714E8
:1004600014F404F40000FF00F7141414141414140A
:10047000F700F7141414171410101F101F1414147D
:10048000F4141010F010F000001F101F0000001FE7
:1004900014000000FC140000F010F01010FF10FF1A
:1004A000141414FF141010101F00000000F010FFAF
:1004B000FFFFFFFFF0F0F0F0F0FFFFFF0000000093
:1004C00000FFFF0F0F0F0F0F3844443844FC4A4A17
:1004D0004A347E02020606027E027E0263554941CC
:1004E000633844443C04407E201E2006027E020203
:1004F00099A5E7A5991C2A492A1C4C7201724C3017
:100500004A4D4D303048784830BC625A463D3E49ED
:100510004949007E0101017E2A2A2A2A2A44445F91
:10052000444440514A444040444A51400000FF0185
:1005300003E080FF000008086B6B08361236243693
:10054000060F090F060000181800000010100030F8
:1005500040FF0101001F01011E00191D1712003C80
:100560003C3C3C000000000000000000230026008E
:100570002900000000080002010000030407000039
:1005800000000000000000000000240027002A00F6
:10059000010204081020408001020408102001021A
:1005A0000408102000000000250028002B0004048F
:1005B000040404040404020202020202030303030B
:1005C0000303292111241FBECFEFD8E0DEBFCDBF2A
:1005D00016E0A0E0B1E0E8E5F0E602C005900D927B
:1005E000A830B107D9F727E0A8E0B6E001C01D9216
:1005F000AC3AB207E1F712E0C2EED2E004C02197B4
:10060000FE010E94992AC13ED107C9F70E94A62186
:100610000C942A300C9400002091E20681E02132F3
:1006200008F044C08091BE068111FCCF8091E106A4
:1006300092E09093BE0691E09093BD069FEF909359
:10064000BC061092BB062093BA06A1ECB6E0EAE91C
:10065000F6E090E0291331C0109299069091990626
:10066000880F892B8093990680919806813049F5EF
:1006700010929806809199068093BB008091BC00EF
:1006800083FDF8CF85EC8093BC008091BE0682305C
:10069000E1F38091BC068F3FB1F08091BC068032BF
:1006A000A1F08091BC06803391F084E01092C006E6
:1006B0001092E2061092BF0608953D9131939F5F1C
:1006C000C9CF85EEE0CF80E0F1CF82E0EFCF83E0CD
:1006D000EDCF8091760690917706891B990B08954E
:1006E0002F923F924F925F926F927F928F929F9242
:1006F000AF92BF92CF92DF92EF92FF920F931F9330
:10070000CF93DF93CDB7DEB7AA970FB6F894DEBFCD
:100710000FBECDBF0D871D8B298F3A8F4B8F5C8FFE
:100720006F8F7BA3FE8EED8EE0915807F0915907F5
:10073000892B21F0E0915A07F0915B07FF27EE0F1C
:10074000FF1FEE0FFF1FE45AF84F60817181828115
:10075000938124E630E040E050E00E94062B522EC8
:10076000632E742E852E962E7A8B898B492E8601C8
:100770007501110FEE08FE2C87019501A6016E2D63
:100780007E2D8E2D9E2D0FE10E94082CA12CEAECCF
:10079000BE2EFAE9CF2EABE3DA2EE12CF12C00E0ED
:1007A00010E00E94332BA52CB62CC72CD82CE92C9A
:1007B000FA880989142D0E949F2A0FE10E94232C98
:1007C00029833A834B835C836D837E838F839887F1
:1007D00029813A814B815C81550F220B322FA9016F
:1007E00029873A874B875C87252D362D472D582D35
:1007F000692D7F2D8989942DA980BA80CB80DC80DA
:10080000E984FE2C0E2D1E2D0E943E2C2983398753
:10081000498B5A8B6B8B7C8B1C016D847D88898CFA
:100820009A8C3C8D3D8B4F8C5BA09301A4016B8D0A
:100830007D89C201211534404B46544F64417105F6
:100840008105910569F060F0612C24E0722E3BE691
:10085000832E44EF942EB4E1BB8F1D8A412C512C82
:10086000EB8DEF8F9301A4016E2F7D89C2012115BD
:1008700038454744584F6D4071058105910560F436
:10088000612C08E5702E87E4882E98EF992E2DE0D4
:100890002F8F1D8A412C512CA980B984C988DA88F0
:1008A000EB88FC8881019301A4016F8D7D89C201D1
:1008B0000E94642B298F3A8F4B8F5C8F2D873E8748
:1008C0004F87588B8D859E85AF85B8891FE0A12EF7
:1008D0000F97A105B10558F02D853E854F855889A4
:1008E0002B35310541055105B8F0BAE5AB2EB12CD9
:1008F000C12CD12CE12CF12C00E010E029813985AC
:1009000049895A896B897C89C1010E949F2A3901D2
:100910004A016F8F7D8B2C01A980B984C988DA8840
:10092000EB88FC8881019301A4016F8D7D89C20150
:100930000E94622BE0E4AE2EF2E4BF2EAFE0CA2E9E
:10094000D12CE12CF12C00E010E00E949F2AA9801C
:10095000B984C988DA88EB88FC8881010E94642BFD
:1009600049014CA35BA3C901DA0121E030E040E07A
:1009700050E00097A105B10521F020E432E44FE0FA
:1009800050E02D8B3E8B4F8B588FBC01CD0127E063
:10099000660F771F881F991F2A95D1F72D893E89E9
:1009A0004F89588D0E94682A29013A016F8F78A3D8
:1009B00089A39AA3A980B984C988DA88EB88FC88BE
:1009C000810194014CA15BA160E070E080E090E0C7
:1009D0000E949F2A2BA33CA34DA35EA36FA378A7DD
:1009E00089A79AA78D859E85AF85B88937E0880F3E
:1009F000991FAA1FBB1F3A95D1F79250A109B109BF
:100A0000840D951DA61DB71DED8DFE8D80839183F0
:100A1000A283B3832F8D38A149A15AA124833583A2
:100A2000468357832D893E894F89588D208731878A
:100A300042875387298D3A8D4B8D5C8D60E070E045
:100A400080E090E00E949F2A29013A014B018987AA
:100A500099838D899E89AF89B88D5C016D01E12CE8
:100A6000F12C00E010E02BA13CA14DA15EA16FA1F3
:100A700078A589A59AA50E94642B59016A017B017A
:100A80008C019201A301B401898599810E943E2CB9
:100A9000AA960FB6F894DEBF0FBECDBFDF91CF91FF
:100AA0001F910F91FF90EF90DF90CF90BF90AF908C
:100AB0009F908F907F906F905F904F903F902F907E
:100AC00008952F923F924F925F926F927F928F92F2
:100AD0009F92AF92BF92CF92DF92EF92FF920F93CD
:100AE0001F93CF93DF93CDB7DEB765970FB6F8941A
:100AF000DEBF0FBECDBF2D833E834F8358876987EE
:100B00007A878B879C87A982BF86C88AD98AEA8A16
:100B1000FB8A0C8B1D8B9E868D86211506ED30077A
:100B200001E140070EE7500703E06007710581050A
:100B3000910511F008F009C12F37304F4A4F52404C
:100B4000610571058105910509F008F469C19501F8
:100B5000A601B7018C899D89A0E00E94532C09F061
:100B60000DC1AD80BE80CF80D884E984FA840B8526
:100B70001C8520E033E245E75EEE64E170E080E052
:100B800090E00E94642BC901DA01A901BD0120FF98
:100B900099C04F5F5F4F6F4F7F4F49835A836B837D
:100BA0007C834F3F51056105710540F08EEF90E069
:100BB000A0E0B0E089839A83AB83BC83E980FA80AC
:100BC0000B811C81A8019701AD80BE80CF80D884A5
:100BD000E984FA840B851C8560E070E080E090E099
:100BE0000E949F2A29013A014B011C01211504E0B2
:100BF00030070BE6400704EF500704E1600771057A
:100C00008105910509F008F47DC089819A81AB8145
:100C1000BC810297A109B10989839A83AB83BC8304
:100C20001C012D010B859101A20160E070E080E0C4
:100C300090E00E949F2A29013A014B011C01898101
:100C40009A81AB81BC819927AA27BB27ED85FE85B8
:100C500080839183A283B3831482158216821782C4
:100C600010861186128613869201A301B401C10178
:100C700065960FB6F894DEBF0FBECDBFDF91CF9162
:100C80001F910F91FF90EF90DF90CF90BF90AF90AA
:100C90009F908F907F906F905F904F903F902F909C
:100CA000089545E050E060E070E01D8286ED8E839F
:100CB00091E19F83AEE7A887B3E0B9871A861B86C8
:100CC0001C8667CF0597A105B10509F066CF16E030
:100CD000E12EF12C00E010E0E982FA820B831C8304
:100CE0006DCF46E057E060E070E0E0E8ED83F0EFC4
:100CF000FE830AEF0F8312E0188719861A861B8677
:100D00001C864BCF2F3F37454744584F6D407105E8
:100D10008105910511F008F092CF89819A81AB810C
:100D2000BC810296A11DB11D89839A83AB83BC83CC
:100D30001C012D01AD80BE80CF80D884E984FA8467
:100D40000B851C8570CF412C63C029813F85488964
:100D500059896A897B898C899D89A0E00E94532CDE
:100D600009F49FCF1D82B6EDBE83E1E1EF83FEE77C
:100D7000F88703E009871A861B861C86AD80BE8033
:100D8000CF80D884E984FA840B851C8529813F852E
:100D9000488959896A897B898C899D890E94622B3F
:100DA00029013A014B011C01A0E00E94532C59F685
:100DB00029813F85488959896A897B898C899D89E0
:100DC0000E94642B022F132F242F352FD901C80125
:100DD0000697A109B109893F9105A105B10508F060
:100DE00043CF10E030E020E0AD85BE850D931D932C
:100DF0002D933C931397FD0114821582168217825E
:100E000018961D921D921D921C921B974424439488
:100E1000512C612C712C812C912C212C312C24CF24
:100E200029813F85488959896A897B898C899D896F
:100E3000A0E00E94532C09F454CF10E81D8380EFEA
:100E40008E839AEF9F83A2E0A887198694CFDF92C2
:100E5000EF92FF920F931F93CF93DF93FC01E080FB
:100E6000F18002811381D481C581B681D780970139
:100E7000A8016D2F7C2F8B2F9D2D285938424C4176
:100E800051096109710981099109273938424C4199
:100E90005105610571058105910509F0D0F49701AF
:100EA000A8016D2F7C2F8B2F9D2D07E00E94082C11
:100EB000208331834283538364837583868397833E
:100EC00087E0DF91CF911F910F91FF90EF90DF901E
:100ED00008959701A8016D2F7C2F8B2F9D2D2053F6
:100EE00031454843510961097109810991092F323E
:100EF000314548435105610571058105910509F0AA
:100F000098F49701A8016D2F7C2F8B2F9D2D06E063
:100F10000E94082C2083318342835383648375832A
:100F20008683978386E0CDCF9701A8016D2F7C2F14
:100F30008B2F9D2D2056324A404751096109710976
:100F4000810991092F35324A4047510561057105E4
:100F50008105910509F098F49701A8016D2F7C2F68
:100F60008B2F9D2D05E00E94082C20833183428326
:100F70005383648375838683978385E0A2CF97012B
:100F8000A8016D2F7C2F8B2F9D2D205C3444414E6A
:100F9000510961097109810991092F3B3444414E7E
:100FA0005105610571058105910509F098F49701D6
:100FB000A8016D2F7C2F8B2F9D2D04E00E94082C03
:100FC000208331834283538364837583868397832D
:100FD00084E077CF9701A8016D2F7C2F8B2F9D2D5B
:100FE00020583948424C51406109710981099109E1
:100FF0002F373948424C51406105710581059105F3
:1010000009F098F49701A8016D2F7C2F8B2F9D2D4F
:1010100003E00E94082C208331834283538364833E
:1010200075838683978383E04CCF9701A8016D2F4A
:101030007C2F8B2F9D2D33514548534061097109F9
:10104000810991092F3F324145485340610571059F
:101050008105910509F098F49701A8016D2F7C2F67
:101060008B2F9D2D02E00E94082C20833183428328
:101070005383648375838683978382E022CF9701AD
:10108000A8016D2F7C2F8B2F9D2D36524A40574043
:1010900061097109810991092F3F35424A40574042
:1010A000610571058105910509F098F49701A80182
:1010B0006D2F7C2F8B2F9D2D01E00E94082C20830B
:1010C000318342835383648375838683978381E06E
:1010D000F8CE80E0F6CE2F923F924F925F926F92C1
:1010E0007F928F929F92AF92BF92CF92DF92EF92B8
:1010F000FF920F931F93CF93DF93CDB7DEB76C971B
:101100000FB6F894DEBF0FBECDBF322E3D87242E22
:101110005E872B013C01A982BF86C88AD98AEA8AE8
:10112000FB8A0C8B1D8B988E8F8A211501EC300762
:101130000AE140070DE3500705E0600771058105EE
:10114000910509F0A0F52F3710EF31071AEF41078D
:1011500012E05107610571058105910509F008F458
:10116000B4C12F3F354D41415E4763407105810554
:10117000910509F008F48FC029813F854889598974
:101180006A897B898C899D89A0E0992493940E9427
:10119000532C09F08EC011E01E8B94E0892E912C07
:1011A000A12CB12C89869A86AB86BC862FC0312CA7
:1011B000B1ECBD872AE1222EEDE3EE8735E0432E28
:1011C000512C612C712CD8CFA32CBD84C22CDE8471
:1011D0007201830120E034E04BE654EF64E170E0FB
:1011E00080E090E00E94642B122FB32FF42FE52FA4
:1011F000A7E00E94532C21F416E0B0E0F0E0E0E01C
:10120000CF011987BA879B87EC871E8A89849A84C5
:10121000AB84BC84A501940160E070E0CB01A32CF9
:10122000BD84C22CDE847201830129833A834B83FF
:101230005C836D837E838F83988760E070E080E0BD
:1012400090E00E949F2A29833F87488B598B6A8BA5
:101250007B8B8C8B9D8B0E89C12CD12C7601C394FA
:1012600040E050E0BA01013009F0A9C0AF89B88D63
:101270001D921D921D921C921397FD0114821582DE
:101280001682178281E090E0A0E0B0E0808791872D
:10129000A287B387DEC029813F85488959896A8939
:1012A0007B898C899D89A0E00E94532C09F48CCF06
:1012B000912CA32CBD84C22CDE8472018301298170
:1012C0003F85488959896A897B898C899D890E94D3
:1012D000642B29873A874B875C8729853A854B851C
:1012E0005C8506E0A02EB12C263031054105510564
:1012F00068F089859A85AB85BC8589309740A105C2
:10130000B105D0F0B8E0AB2E17E0B12EC12CD12C36
:10131000E12CF12C00E010E029813F8548895989B2
:101320006A897B898C899D890E94642B322E3D8736
:10133000242E5E872B013C01A32CBD84C22CDE84AD
:101340007201830129813F85488959896A897B898E
:101350008C899D890E94622BE0E4AE2EF2E4BF2EC0
:10136000AFE0CA2ED12CE12CF12C00E010E00E945D
:101370009F2AA32CBD84C22CDE84720183010E94AB
:10138000642BA32FF42FE52F422F5A2F6F2F7E2F80
:10139000A0E4CA2EA2E4DA2EAFE0EA2EF12C411529
:1013A00051056105710521F4C12CD12C7601C3943E
:1013B000AA24A3949A1409F46DC001E00E8BCB010A
:1013C000BA0117E0660F771F881F991F1A95D1F78A
:1013D000A70196010E94682A298F3A8F4B8F5C8F54
:1013E00089849A84AB84BC8407E0880C991CAA1C6D
:1013F000BB1C0A95D1F795018401125021093109CE
:1014000048015901298D3A8D4B8D5C8D280D391D70
:101410004A1D5B1DAF89B88D2D933D934D935C9311
:101420001397FD0164837583868397831896CD9205
:10143000DD92ED92FC921B978E88882051F03982C4
:101440009D849F86288AAE84A98A4A8A5B8A6C8A90
:101450007D8A29813F85488959896A897B898C8958
:101460009D896C960FB6F894DEBF0FBECDBFDF919D
:10147000CF911F910F91FF90EF90DF90CF90BF9091
:10148000AF909F908F907F906F905F904F903F9024
:101490002F900895AF89B88D1D921D921D921C92B8
:1014A0001397FD01148215821682178281E090E065
:1014B000A0E0B0E080879187A287B3873982FD855D
:1014C000FF87288A8E84898AC0CF29813F854889F1
:1014D00059896A897B898C899D89A0E0E0E83E2E44
:1014E000F0EFFD87FAEF2F2E02E00E87412C512CF2
:1014F000612C712C0E94532C09F0DACE18E0B7E071
:101500007DCEDF92EF92FF920F931F93CF93DF93E5
:10151000FC01E080F18002811381D481C581B68114
:10152000D7809701A8016D2F7C2F8B2F9D2D2058E0
:101530003A414640510961097109810991092F37E2
:101540003A4146405105610571058105910509F053
:10155000D0F49701A8016D2F7C2F8B2F9D2D07E0D4
:101560000E94082C208331834283538364837583D4
:101570008683978387E0DF91CF911F910F91FF9032
:10158000EF90DF9008959701A8016D2F7C2F8B2F8E
:101590009D2D35534C40510961097109810991090B
:1015A0002F3F34434C40510561057105810591057C
:1015B00009F098F49701A8016D2F7C2F8B2F9D2D9A
:1015C00006E00E94082C2083318342835383648386
:1015D00075838683978386E0CECF9701A8016D2F10
:1015E0007C2F8B2F9D2D3A56484151096109710975
:1015F000810991092F3F394648415105610571051F
:101600008105910509F098F49701A8016D2F7C2FB1
:101610008B2F9D2D05E00E94082C2083318342836F
:101620005383648375838683978385E0A4CF970172
:10163000A8016D2F7C2F8B2F9D2D345D40435109C8
:1016400061097109810991092F3F334D40435105CB
:10165000610571058105910509F098F49701A801CC
:101660006D2F7C2F8B2F9D2D04E00E94082C208352
:10167000318342835383648375838683978384E0B5
:101680007ACF9701A8016D2F7C2F8B2F9D2D385A73
:101690004146510961097109810991092F3F374A72
:1016A00041465105610571058105910509F098F4E0
:1016B0009701A8016D2F7C2F8B2F9D2D03E00E9499
:1016C000082C20833183428353836483758386830C
:1016D000978383E050CF9701A8016D2F7C2F8B2F2C
:1016E0009D2D3055434C51096109710981099109BA
:1016F0002F3F3F44434C510561057105810591051C
:1017000009F098F49701A8016D2F7C2F8B2F9D2D48
:1017100002E00E94082C2083318342835383648338
:1017200075838683978382E026CF9701A8016D2F6A
:101730007C2F8B2F9D2D305A4648514061097109ED
:10174000810991092F3F3F49464851406105710584
:101750008105910509F098F49701A8016D2F7C2F60
:101760008B2F9D2D01E00E94082C20833183428322
:101770005383648375838683978381E0FCCE80E006
:10178000FACE0895089528E030E040E8E0919B0704
:10179000F0919C0750819091A2079095952390839A
:1017A000E0919907F0919A079091A107582F54233F
:1017B00089F05081952B9083E0919B07F0919C07D5
:1017C00090815091A207952B908346952150310925
:1017D000E9F60895508190959523EDCFAF92BF9291
:1017E000CF92DF92EF92FF920F931F93CF93DF93ED
:1017F0006C017B018B01040F151FEB015E01AE181C
:10180000BF08C017D10759F06991D601ED91FC913D
:101810000190F081E02DC6010995892B79F7C5016A
:10182000DF91CF911F910F91FF90EF90DF90CF90BC
:10183000BF90AF900895833081F028F4813099F003
:101840008230A9F008958730A9F08830C9F084303B
:10185000B1F4809180008F7D03C0809180008F77EC
:1018600080938000089584B58F7784BD089584B5F2
:101870008F7DFBCF8091B0008F778093B00008956B
:101880008091B0008F7DF9CFCF93DF93282F30E088
:10189000F901EE58FA4F8491F901E057FA4FD491CB
:1018A000F901E255FA4FC491CC23A1F081110E94B5
:1018B0001B0CEC2FF0E0EE0FFF1FE859FA4FA5913B
:1018C000B491EC91ED2381E090E009F480E0DF91A8
:1018D000CF91089580E090E0FACF1F93CF93DF93EC
:1018E000282F30E0F901EE58FA4F8491F901E057C2
:1018F000FA4FD491F901E255FA4FC491CC23A9F0E3
:10190000162F81110E941B0CEC2FF0E0EE0FFF1F31
:10191000EC55FA4FA591B4918FB7F894EC91111151
:1019200008C0D095DE23DC938FBFDF91CF911F914C
:101930000895DE2BF8CF109277061092760610925B
:10194000C0061092E2061092BE0681E08093BD06AA
:101950001092980661E082E10E946D0C61E083E1E3
:101960000E946D0CE9EBF0E080818E7F80838081A6
:101970008D7F808388E48093B80085E48093BC00E9
:1019800081EC9BE0909375068093740682EC9BE05B
:1019900090937306809372060895CF93DF9390E03F
:1019A000FC01E057FA4F249182559A4FFC01849133
:1019B0008823C9F090E0880F991FFC01EA57FA4F7D
:1019C000A591B491FC01EC55FA4FC591D4916111E8
:1019D0000DC09FB7F8948C91209582238C938881B9
:1019E000282328839FBFDF91CF910895623051F45F
:1019F0009FB7F8943C91822F809583238C93E88144
:101A00002E2BEFCF8FB7F894EC912E2B2C938FBF0A
:101A1000EACF3FB7F8948091540690915506A09173
:101A20005606B091570626B5A89B05C02F3F19F062
:101A30000196A11DB11D3FBFBA2FA92F982F88274E
:101A4000BC01CD01620F711D811D911D42E0660F29
:101A5000771F881F991F4A95D1F708958F929F92FB
:101A6000AF92BF92CF92DF92EF92FF924B015C0157
:101A70000E94090D6B017C010E94090D6C197D0902
:101A80008E099F09683E734081059105A8F321E006
:101A9000821A9108A108B10888EEC80E83E0D81E0A
:101AA000E11CF11C81149104A104B10429F7FF90F9
:101AB000EF90DF90CF90BF90AF909F908F90089560
:101AC0002FB7F8946091500670915106809152069C
:101AD000909153062FBF08950F931F93CF93DF93D9
:101AE000EC018E89823009F453C0833009F4ACC014
:101AF000813009F05CC0EC81FD81E41BF50BAF0186
:101B0000421B530B77FD3FC08E819F816817790779
:101B1000D4F557FF04C0240F351F50E040E08C81FE
:101B20009D81FA01E20FF31F8E179F071CF49C01A1
:101B3000241B350B1216130634F5FB0177FD37967F
:101B4000A3E0F595E795AA95E1F7F695FE2FEE2728
:101B5000F795E795E40FF51FEF5FFE4F6770772766
:101B600081E090E001C0880F6A95EAF7482F0130C4
:101B7000110509F472C008F47CC02E0F3F1F02301B
:101B8000110509F483C0DF91CF911F910F91089542
:101B9000AC81BD81CD01861B970BBC0161507109E1
:101BA000EE81FF81E41BF50BAF01421B530B77FD68
:101BB000EACF8C819D81681779072CF757FF04C005
:101BC000240F351F50E040E08E819F81FA01E20F23
:101BD000F31F8E179F071CF49C01241B350B121654
:101BE00013068CF6922FA42FA695A695A69580E8AD
:101BF000A89FD0011124A60FB71FAF5FBE4F47703B
:101C000009F457C058E0541B452F652F70E0FB01C5
:101C1000E95DFA4F8081251708F0B0C0621B710999
:101C20002FEF30E002C0359527956A95E2F78223C1
:101C300001301105A9F108F464C00230110509F062
:101C4000A2CF2C9182272EC0AE81BF81CD01861BF1
:101C5000970BBC016150710955CF2E0F3F1FE21742
:101C6000F30709F490CF8191DF011197842B8C93B6
:101C7000F6CF80952E0F3F1FE217F30709F483CFAD
:101C80009191DF01119798239C93F6CFE217F30708
:101C900009F479CF8191DF01119784278C93F6CFD6
:101CA0002C91822B8C93941708F46DCF941BA05821
:101CB000BF4F983008F447C00230110531F5FD01DF
:101CC000892F208120952083E058FF4F885088304D
:101CD000C0F728EF290F26952695269530E02F5F2F
:101CE0003F4F3695322F222737952795A20FB31FE6
:101CF000977009F448CFE92FF0E0E15EFA4F808158
:101D000032C080952C918223CDCF81E00130110526
:101D100009F080E08195FD01292F8083E058FF4F75
:101D200028502830D0F728EF290F2695269526959C
:101D300030E02F5F3F4F3695322F2227379527957A
:101D4000A20FB31F9770992309F41DCFE92FF0E07C
:101D5000E15EFA4F80810130110541F058F0023008
:101D6000110509F010CF9C91892702C09C91892B05
:101D70008C9309CF80959C918923FACF013011056E
:101D800009F48ECF08F4BDCF0230110509F459CF04
:101D90008DCF0F931F93CF93DF93EC018E89823009
:101DA00009F45EC0833009F4B5C0813009F067C022
:101DB000AC81BD81CD01841B950BAC014150510913
:101DC00057FD49C08C819D81481759070CF043C0CD
:101DD00077FF04C0260F371F70E060E08E819F817F
:101DE000FB01E20FF31F8E179F071CF49C01261BBB
:101DF000370B121613067CF5922FA62FA695A695E3
:101E0000A69580E8A89FD0011124A40FB51FAF5F4D
:101E1000BE4F677009F48FC048E0461B642F70E026
:101E2000FB01E95DFA4F8081241708F002C1621BB3
:101E300071092FEF30E002C0359527956A95E2F7DA
:101E400082230130110509F46DC008F49CC00230F2
:101E5000110509F4F8C0DF91CF911F910F910895FA
:101E6000EC81FD81E61BF70BAE81BF81CD01841BA8
:101E7000950BAC0141505109BF01621B730B57FD1B
:101E8000EACF8E819F81481759072CF777FF04C04E
:101E9000260F371F70E060E08C819D81FB01E20F0F
:101EA000F31F8E179F071CF49C01261B370B12167D
:101EB00013068CF6FA0157FD379693E0F595E795F2
:101EC0009A95E1F7F695FE2FEE27F795E795E60F41
:101ED000F71FEF5FFE4F4770552781E090E001C08C
:101EE000880F4A95EAF7482F0130110509F488C098
:101EF00008F492C02E0F3F1F0230110509F0ABCF3E
:101F0000E217F30709F4A7CF8191DF011197842726
:101F10008C93F6CFEE81FF81E61BF70BBF01621BAE
:101F2000730B4ECF2C91822B8C93941708F493CF84
:101F3000941BA058BF4F983008F447C002301105D9
:101F400031F5FD01892F208120952083E058FF4F36
:101F500088508830C0F728EF290F269526952695BA
:101F600030E02F5F3F4F3695322F22273795279548
:101F7000A20FB31F977009F46ECFE92FF0E0E15E76
:101F8000FA4F808132C080952C918223CDCF81E0A1
:101F90000130110509F080E08195FD01292F808332
:101FA000E058FF4F28502830D0F728EF290F26950A
:101FB0002695269530E02F5F3F4F3695322F22270A
:101FC00037952795A20FB31F9770992309F443CF34
:101FD000E92FF0E0E15EFA4F80810130110541F018
:101FE00058F00230110509F036CF9C91892702C0C4
:101FF0009C91892B8C932FCF80959C918923FACF2C
:102000002E0F3F1FE217F30709F425CF8191DF015F
:102010001197842B8C93F6CF80952E0F3F1F2E1790
:102020003F0709F418CF9191DF01119798239C93F2
:10203000F6CF0130110509F475CF08F4A4CF0230B2
:10204000110509F075CF2C9182276ECFDC0177FD49
:1020500067C018968D919C911997681779070CF0B5
:102060005FC057FD5DC01A968D919C911B974817D4
:1020700059070CF055C056968C9156978230B9F09E
:10208000833041F1813049F414968D919C91841BE9
:10209000950BAB01BC01615071092130310521F173
:1020A00008F43FC02230310509F458C00895149651
:1020B000ED91FC911597E61BF70BBF01615071097B
:1020C00016968D919C91FC01E41BF50BAF014150DC
:1020D0005109E3CF16968D919C91861B970BBA01FF
:1020E000AC0141505109D9CFFA0157FD3796A3E011
:1020F000F595E795AA95E1F7F695FE2FEE27F7956A
:10210000E795E60FF71FEF5FFE4F4770552721E079
:1021100030E001C0220F4A95EAF78081822B80834C
:102120000895FA0157FD379623E0F595E7952A952E
:10213000E1F7F695FE2FEE27F795E795E60FF71FE7
:10214000EF5FFE4F4770552781E090E001C0880F98
:102150004A95EAF7809590818923E1CFFA0157FDEE
:10216000379683E0F595E7958A95E1F7F695FE2F8A
:10217000EE27F795E795E60FF71FEF5FFE4F4770E5
:10218000552721E030E001C0220F4A95EAF780810F
:102190008227C5CF0895FC016370668B8481958189
:1021A00026813781613039F0633029F0918780874B
:1021B0003387228708953187208793878287089500
:1021C0002F923F924F925F926F927F928F929F9247
:1021D000AF92BF92CF92DF92EF92FF920F931F9335
:1021E000CF93DF93CDB7DEB76A970FB6F894DEBF13
:1021F0000FBECDBF9A8F898F7A8369834A01D22E11
:1022000018870F833701BC2CDC0159962D913C9126
:102210005A972115310509F015C118968D919C9199
:102220001997681779070CF0D7C11A968D919C9170
:10223000481759070CF0D0C14C2C512CB6E0CB9E5E
:10224000600D711D11247C876B87161617060CF024
:10225000C3C1EA2DF0E0FA87E98793E0EE0FFF1F94
:102260009A95E1F7F88BEF87CF01840F951F181629
:1022700019060CF0B1C1A98DBA8D58968C918111B7
:1022800004C0BFEABD1508F4D394A98DBA8DED91B1
:10229000FC9111970284F385E02DCD010995B5E0FD
:1022A000DB9EC0011124E981FA81FC83EB83312C90
:1022B000212C9C0128593F4F388F2F8B4A2D50E0FD
:1022C0005E8B4D8BEF89F88DE20DF31D44919E825C
:1022D0008D82D12CC12C69817A81620D731D7A8B1C
:1022E000698B842F90E09C8B8B8BE98DFA8DA0817C
:1022F000B18140FF82C0F1E0BF126FC0AF126DC06C
:102300001C96ED91FC912F813885A4014C0D5D1D2B
:1023100069897A89898D9A8D0995EB89FC89F5956A
:10232000E7954E2F5FEFC51AD50A6D817E818D89A5
:102330009E89680F791F7E836D8398E0C916D1044A
:1023400081F6AFEF2A1A3A0AEB81FC81E40DF51D04
:10235000FC83EB83F5E02F16310409F0B3CF2F8116
:10236000388526153705B9F0A98DBA8DED91FC9108
:10237000B1E0BB1257C0AB1255C069817A816B5F67
:102380007F4F0088F189E02D830128E030E0A4012F
:10239000898D9A8D0995A98DBA8DED91FC91119732
:1023A0000688F789E02DCD016A960FB6F894DEBF56
:1023B0000FBECDBFDF91CF911F910F91FF90EF9096
:1023C000DF90CF90BF90AF909F908F907F906F9055
:1023D0005F904F903F902F9009941E96ED91FC9145
:1023E000EF80F88409851A8592014D815E816B81A9
:1023F0007C81898D9A8D099590CF2F8138852615FE
:10240000370509F48ACF31E0B31207C0A31205C023
:102410001C96ED91FC91930178CF1E96ED91FC9165
:102420007301E0CF6B857C85641975090684F78597
:10243000E02D73010F8518899201A401898D9A8D71
:102440000995A9CFF9013496949132974591549109
:10245000D91AB7E0DB9E400D511D1124F9012591D9
:1024600034913C8B2B8BFA0125903490FA013296F3
:10247000749031963491398B3296649031964490B1
:1024800041E04C1518F04A1508F07FC0662D062C67
:10249000000C770B7C836B83842D042C000C990B30
:1024A0009E838D83A98DBA8DED91FC911197028445
:1024B000F385E02DCD010995512CD12CC12CEA2DAD
:1024C000F0E0FA87E9872B2D30E03C872B87A401C9
:1024D000440D511D47FC5A95588F4F8B69817A8165
:1024E000660D711D67FC7A957E876D877989C716A1
:1024F00008F051CF2C2D30E04D815E81420F531FEB
:10250000A985BA854A9FC0014B9F900D5A9F900D97
:102510001124FC01E80DF91DF88BEF87852D612C46
:102520004F89588D420F531F5E8B4D8B671408F0F7
:1025300050C044244394480E877041F4C101019671
:10254000EB89FC89E20DF31DD4901C01D7FE19C064
:10255000A98DBA8DED91FC91662D70E0B1E0BB12B2
:1025600019C0AB1217C02D853E85620F731F0484FE
:10257000F585E02D2F8138854D895E89898D9A8D6D
:102580000995DD0C6394842DD1CF1E821D821C829F
:102590001B8288CF4B815C81640F751FAB85BC8526
:1025A0006A9FC0016B9F900D7A9F900D11246981E5
:1025B0007A81680F791F0684F785E02DEF80F88413
:1025C00009851A859D014F855889898D9A8D0995B0
:1025D000D8CF570CC3948ACF6A960FB6F894DEBF53
:1025E0000FBECDBFDF91CF911F910F91FF90EF9064
:1025F000DF90CF90BF90AF909F908F907F906F9023
:102600005F904F903F902F9008958F929F92AF923E
:10261000CF92EF92FF920F931F93CF93DF93EC0132
:10262000262F898D9A8D009709F051C06A30D1F418
:102630001D861C868D8948E0849F900111248E851B
:102640009F85820F931F9F878E8781E090E0DF91A7
:10265000CF911F910F91FF90EF90CF90AF909F90EF
:102660008F9008956D3089F3CC88AD888F89882349
:10267000C1F08C859D8536E0C39E800D911D11248F
:10268000488559854817590764F44E855F851D862E
:102690001C8638E0A39EC0011124840F951F9F87DC
:1026A0008E87EA88FB88088919894E855F856C8545
:1026B0007D85CE010E94E0102C898C859D8546E0A9
:1026C000249F800D911D11249D878C87BECF6A3079
:1026D00069F41D861C86FC013896E4912D898E854F
:1026E0009F85E29F800D911D1124ADCF6D3009F4BF
:1026F000ACCFFC0134963491631708F4A6CF329620
:10270000E491E61708F4A1CFFC01329685909490ED
:10271000462F431B342F47E0349F800C911C11241B
:10272000F401329634913196E4913323A9F1EE23EA
:1027300099F1CC88F4013596E491AD884F89442312
:1027400001F10E2E000CFF0BE30FF11DCE9EA00138
:10275000CF9E500D11246C857D85460F571F6885CF
:102760007985641775076CF44E855F851D861C8618
:10277000FC013896E491AE9E400D511D11245F87F7
:102780004E87EA88FB88088919894E855F856C85A4
:102790007D85CE010E94E010F4013496E4912C89ED
:1027A0008C859D85E29F800D911D11248DCF6F92A8
:1027B0007F928F929F92AF92BF92CF92DF92EF92D1
:1027C000FF920F931F93CF93DF93EC016B015A019C
:1027D00039014801E881F9810284F385E02D0995EA
:1027E000E881F9810288F389E02D87019301A50131
:1027F000B601CE010995A501480D591D4150510959
:10280000E881F9810288F389E02D9301B601CE01B8
:102810000995E881F9810088F189E02D9401A501ED
:10282000B601CE010995C60CD71CB60161507109DD
:10283000E881F9810088F189E02D9401A501CE019C
:102840000995E881F9810688F789E02DCE01DF91AD
:10285000CF911F910F91FF90EF90DF90CF90BF909D
:10286000AF909F908F907F906F9009946F927F921E
:102870008F929F92AF92BF92CF92DF92EF92FF9290
:102880000F931F93CF93DF935C01EB016A01490122
:1028900038018701DC01ED91FC916217730719F58E
:1028A000641675062CF0962D872D3A01C92ED82E68
:1028B0009601261937092F5F3F4F048CF58DE02DC7
:1028C000A301BE01C5010995DF91CF911F910F9121
:1028D000FF90EF90DF90CF90BF90AF909F908F9040
:1028E0007F906F9008954615570591F42617370786
:1028F00024F0892D4B01C22FD82F9E0128193909A8
:102900002F5F3F4F068CF78DE02DA601B401DACF83
:102910000284F385E02D0995D501ED91FC910488A1
:10292000F589E02D83019401A601BE01C501099539
:10293000D501ED91FC910688F789E02DC501DF9165
:10294000CF911F910F91FF90EF90DF90CF90BF90AC
:10295000AF909F908F907F906F900994EF92FF922D
:102960000F931F93DC011A960D911C911B971896DB
:102970002D913C911997ED91FC9100A0F1A1E02DD2
:102980007B0150E040E070E060E009951F910F91FD
:10299000FF90EF9008954F925F926F927F928F9287
:1029A0009F92AF92BF92CF92DF92EF92FF920F93DE
:1029B0001F93CF93DF936C012B015A01390148011A
:1029C000DC01ED91FC910284F385E02D0995E20193
:1029D000640C751CD601ED91FC91C615D7055CF40D
:1029E0000088F189E02D87019401A501BE01C6018F
:1029F00009952196EFCF0688F789E02DC601DF9172
:102A0000CF911F910F91FF90EF90DF90CF90BF90EB
:102A1000AF909F908F907F906F905F904F900994B0
:102A20008F929F92AF92BF92CF92DF92EF92FF92DE
:102A30000F931F93CF93DF93EC015B014A01690170
:102A4000E881F9810284F385E02D099595012C0D2B
:102A50003D1D21503109E881F9810488F589E02D77
:102A600078018401A401B501CE010995E881F981BD
:102A70000688F789E02DCE01DF91CF911F910F914C
:102A8000FF90EF90DF90CF90BF90AF909F908F908E
:102A900009948F929F92AF92BF92CF92DF92EF9262
:102AA000FF920F931F93CF93DF93EC015B014A01D9
:102AB00069017801E881F9810284F385E02D0995A7
:102AC000C80CD91C860101501109E881F9810488DC
:102AD000F589E02D9501A401B501CE010995E881A4
:102AE000F9810688F789E02DCE01DF91CF911F9102
:102AF0000F91FF90EF90DF90CF90BF90AF909F909D
:102B00008F9009940895EF92FF920F931F93DC0129
:102B1000ED91FC9100A0F1A1E02D09951F910F917D
:102B2000FF90EF9008950F931F93DC01ED91FC91BE
:102B3000068CF78DE02D09951F910F9108950F9345
:102B40001F93DC01ED91FC91048CF58DE02D09952E
:102B50001F910F910895DC01ED91FC910084F185A6
:102B6000E02D09942F923F924F925F926F927F9245
:102B70008F929F92AF92BF92CF92DF92EF92FF928D
:102B80000F931F93CF93DF9300D000D000D0CDB729
:102B9000DEB73C016A013E832D83FC82EB82580143
:102BA000A41AB50AB7FE03C0B194A194B1088D80F0
:102BB0009E80861A970A97FE03C09194819491088B
:102BC0008A149B045CF0902F812F0D811E819D83C0
:102BD0008E839C2D8D2D6B01692F782F0C151D0573
:102BE0005CF09D818E817E836D83692F782F902F7D
:102BF000812F8601C92ED82E1601201A310A2B01E9
:102C00002D813E81421A530A57FE03C051944194CC
:102C10005108710137FE03C03FEFE31AF30AF59440
:102C2000E7948D819E81861797075CF5A1E0B0E05F
:102C3000BA83A983C016D1064CF1D301ED91FC9162
:102C40000484F585E02D2B813C81A8016D817E8176
:102C50008A149B041CF04D815E81B801C301099563
:102C6000E418F508F7FE0AC02D813E8189819A811A
:102C7000280F391F3E832D83E20CF31C0F5F1F4F7B
:102C8000D9CF2FEF3FEF3A832983D4CF26960FB6C3
:102C9000F894DEBF0FBECDBFDF91CF911F910F9192
:102CA000FF90EF90DF90CF90BF90AF909F908F906C
:102CB0007F906F905F904F903F902F900895089570
:102CC00085ED8093BC008091BC0084FDFCCF109208
:102CD000BE06089520912C06260F3327331F21327C
:102CE0003105ECF42091BE06FC0190E080E0243038
:102CF00069F082E00895A0912C062191AC01445F17
:102D0000594FA40FB52FB11D2C930196861798F338
:102D100080912C06680F60932C0680E0089581E076
:102D20000895E091770680917606E81730F4F0E098
:102D3000E858F94F808190E008958FEF9FEF089554
:102D400090917706809176062FEF3FEF981748F421
:102D5000E92FF0E0E858F94F208130E09F5F909331
:102D60007706C9010895CF92DF92EF92FF920F93F9
:102D70001F93CF93DF937C01CB018A012091BF0683
:102D8000222389F0EB016B01C40ED51ECC15DD05A5
:102D900069F06991D701ED91FC910190F081E02DEE
:102DA000C7010995F3CF642F0E946A16C801DF910D
:102DB000CF911F910F91FF90EF90DF90CF900895EA
:102DC000CF93DF931F92CDB7DEB769832091BF0603
:102DD0002223F9F02091E206203258F021E030E081
:102DE000FC013383228390E080E00F90DF91CF914C
:102DF00008958091C006E82FF0E0EF53F94F9981D4
:102E000090838F5F8093C0068093E20681E090E01C
:102E1000ECCF61E0CE0101960E946A16F7CFCF9306
:102E2000C62F90916D0721E02093BF069093E10695
:102E30001092C0061092E206682F83EE96E00E9480
:102E4000E0166C2F83EE96E00E94E016CF910C9472
:102E50000C03EF92FF920F931F93CF93DF93062FF4
:102E60007A0190916D0721E02093BF069093E106CF
:102E70001092C0061092E206682F83EE96E00E9440
:102E8000E016E70110E0CE018E199F098017910727
:102E900034F4699183EE96E00E94E016F4CFDF915E
:102EA000CF911F910F91FF90EF900C940C03CF9353
:102EB000C82F809193078F3FB1F1E0919D07F0916A
:102EC0009E0780819091A307892B8083E0919F07C3
:102ED000F091A00790818091A40780958923808339
:102EE000E0919D07F0919E0790818091A3078095C6
:102EF0008923808380919807882389F0CEBD0000C4
:102F00000DB407FEFDCF8EB5E0919D07F0919E07B1
:102F100080819091A307892B8083CF9108958C2F76
:102F20000E94C30BF1CF8091910791E09093BF066F
:102F30008093E1061092C0061092E20660E083EEF4
:102F400096E00E94E0166C2F83EE96E00E94E01659
:102F5000CF910C940C038F929F92AF92BF92CF921D
:102F6000DF92EF92FF920F931F93CF93DF9380E056
:102F70000E94571780E10E94571780E40E9457175C
:102F8000809193078F3F09F46BC030EBF32ED0E0B4
:102F9000C0E08F2D0E94571782E00E94571780E1F2
:102FA0000E94571710E000E0CE018F5F9E4F6C012A
:102FB000E0919D07F0919E0780819091A307892B56
:102FC0008083E0919F07F091A00780819091A407F2
:102FD000892B8083E0919D07F0919E0790818091DD
:102FE000A3078095892380835601A00EB11E20E19E
:102FF000E22EF50181915F0190919807992369F183
:103000008EBD00000DB407FEFDCF8EB5EA94E11031
:10301000F0CFE0919D07F0919E0780819091A307EA
:10302000892B8083005F1F4F0038110509F0C0CF46
:10303000C058DF4FF394C115F4E0DF0709F0A9CFC2
:10304000DF91CF911F910F91FF90EF90DF90CF9084
:10305000BF90AF909F908F9008950E94C30BD6CFE2
:103060009090B8008CE08093B80090EBF92ED0E0FF
:10307000C0E0882483948F2D0E94571782E00E941D
:10308000571780E10E94571710E000E0CE018F5FD4
:103090009E4F5C01809191078092BF068093E1066C
:1030A0001092C0061092E20660E483EE96E00E9461
:1030B000E0166501C00ED11E80E1E82EF601619197
:1030C0006F0183EE96E00E94E016EA94E110F6CFDD
:1030D0000E940C03005F1F4F00381105D9F6C0583D
:1030E000DF4FF394C115F4E0DF0729F69092B800A2
:1030F000A7CF90E080E0089580915A068230C9F011
:1031000018F4813031F008958330D9F0843009F11A
:10311000089582E080935A0684E690E0A0E0B0E053
:103120008093080690930906A0930A06B0930B06B5
:10313000089583E080935A0688EE93E0A0E0B0E023
:10314000EFCF84E080935A0680E197E2A0E0B0E000
:10315000E7CF81E080935A0680EA96E8A1E0B0E0EC
:10316000DFCF0F931F93409108065091090660919D
:103170000A0670910B0681309105A1F400916A0650
:1031800010916B0620916C0630916D06040F151F8F
:10319000261F371F00936A0610936B0620936C0658
:1031A00030936D0600916A0610916B0620916C06B3
:1031B00030916D0600341A4329463D4060F000E42A
:1031C0001AE329E63DE000936A0610936B0620930C
:1031D0006C0630936D068F3F9807A1F400916A0644
:1031E00010916B0620916C0630916D06041B150B37
:1031F000260B370B00936A0610936B0620936C0620
:1032000030936D0600916A0610916B0620916C0652
:1032100030916D064034E2E45E07EFE06E07710521
:1032200069F5013412442F40310540F440936A0699
:1032300050936B0660936C0670936D068130910518
:1032400029F4209100012F5F2093000120910001BB
:103250002B32F0F021E020930001019661F480917F
:10326000000181508093000180910001811103C011
:103270008AE2809300011F910F9108950031174257
:1032800021053105D8F640E157E260E070E0CECF8D
:10329000019651F7E4CFCF9390916D0721E02093F1
:1032A000BF069093E1061092C0061092E206682FC6
:1032B00083EE96E00E94E0160E940C0380916D0759
:1032C0009091BE069111FCCF91E09093BE061092B2
:1032D000BD062FEF2093BC061092BB061092BA06D3
:1032E0009093990690919906880F892B809399065F
:1032F00080919806813061F5109298068091990628
:103300008093BB008091BC0083FDF8CF85EC809357
:10331000BC008091BE068130E1F38091BB06811133
:1033200019C08091BB06EAE9F6E0A8E7B6E0C0E084
:10333000C81312C010927706C093760680E0909171
:103340007706C91769F083EE96E00E94A016F7CFC2
:1033500085EEDDCF81E0E7CF91919D93CF5FE8CF00
:10336000CF9108951F93CF93DF93C62F142F815DC4
:103370009A4FFC01D0818D2F0E944B198378111137
:103380008C60F0E1CF9FB0011124682B8D2FDF916D
:10339000CF911F910C940F17CF93DF93D62FC0E1DD
:1033A000C80F8C2F0E944B19682FD13031F4606404
:1033B0008C2FDF91CF910C940F176F7BF9CFCF93A8
:1033C000DF93D82FC62F83E00E944B1961E070E095
:1033D00001C0660FDA95EAF7C13039F460956823C9
:1033E00083E0DF91CF910C940F17682BF9CFFF92F8
:1033F0000F931F93CF93DF93EC018B01F82E80E1A5
:10340000F80E8F2D0E944B19682F0115110581F4BC
:103410006F7D8F2D0E940F17CC0FDD1FC151D94F2B
:103420001A870987DF91CF911F910F91FF9008951F
:103430006062EFCFE0915906E150E53130F5F0E000
:10344000EC5DF54E0C94992A391A4E1A531A581AF3
:103450009E1A451A5D1A621A671A6C1A711A761A40
:103460007B1A801A851A8A1A8F1A941A991A9E1A28
:10347000A31A80ED91EBA7E3B0E080936A069093E6
:103480006B06A0936C06B0936D0660E281EB0E9420
:103490000F1782E080935A060C947C1880E696E51C
:1034A000ACE6B0E0EACF88E19BE4A8EDB0E0E5CF80
:1034B00080EA9AEFA8EBB1E0E0CF80E09DEDADE6C9
:1034C000B0E0DBCF80E896E9A8E9B0E0D6CF80EAAB
:1034D0009FEBA3EBB0E0D1CF80E39AEFAFECB0E08D
:1034E000CCCF80E296E2A7EDB0E0C7CF80EC91EEC2
:1034F000A4EEB0E0C2CF88ED94E6ADE0B1E0BDCF80
:1035000088E092E7A8E4B1E0B8CF88E597E3ACE9BA
:10351000B1E0B3CF80E899E5A1EBB1E0AECF80E8B0
:1035200090EFAAEFB2E0A9CF80E091EEA5EFB5E071
:10353000A4CF80E894EAAFEBB7E09FCF80E094E4BB
:10354000A5E9B8E09ACF80E09FEEACE1BDE095CF71
:103550002F923F924F925F926F927F928F929F92A3
:10356000AF92BF92CF92DF92EF92FF920F931F9391
:10357000CF93DF93CDB7DEB72D970FB6F894DEBFAC
:103580000FBECDBF3C01C982DA82EB82FC820D8383
:103590001E832F83388749875A876B877C87BAA019
:1035A0003C2C2D2C5E2C0D87412E922EC984DA8462
:1035B000EB84FC8484E190E00E945F2C8C01FC0190
:1035C000D082C182862D880F880F880F845D0E946B
:1035D0004B19F52DF3705F2E8C7F582AF80152821B
:1035E000238234828CE0F694E794D794C7948A952A
:1035F000D1F7FC2DF07FCF2E892D8F70C82AF801CE
:10360000C58246828D85878393E06916710409F42B
:103610006CC0A8F5F1E06F16710409F448C082E0AF
:103620006816710409F452C0A80168E08AE20E9499
:1036300029176A2D90E080E00E94CC194B2D682D4F
:1036400090E080E00E94B219C8012D960FB6F89460
:10365000DEBF0FBECDBFDF91CF911F910F91FF90C5
:10366000EF90DF90CF90BF90AF909F908F907F9022
:103670006F905F904F903F902F900C94FB2C94E0B4
:103680006916710409F440C0E5E06E16710461F634
:10369000A80168E082E50E9429176A2D85E090E084
:1036A0000E94CC194B2D682D85E090E0CBCFA8016E
:1036B00068E082E30E9429176A2D81E090E00E9471
:1036C000CC194B2D682D81E090E0BCCFA80168E0BB
:1036D0008AE30E9429176A2D82E090E00E94CC19AB
:1036E0004B2D682D82E090E0ADCFA80168E082E428
:1036F0000E9429176A2D83E090E00E94CC194B2D7F
:10370000682D83E090E09ECFA80168E08AE40E94E3
:1037100029176A2D84E090E00E94CC194B2D682D6A
:1037200084E090E08FCF2F923F924F925F926F9202
:103730007F928F929F92AF92BF92CF92DF92EF9241
:10374000FF920F931F93CF93DF93CDB7DEB72E97E2
:103750000FB6F894DEBF0FBECDBF19013A014B0181
:103760008D879E872801012B09F073C0E0915807CF
:10377000F0915907EE0FFF1FEE0FFF1FEC59F84FA6
:10378000A080B180C280D380CE0101967C018901E6
:103790009301AB016D857E8590E080E00E9470030F
:1037A00084E190E00E945F2C8C0189859A85AB852D
:1037B000BC85F8019083818339814A812B812370F4
:1037C0002283438334832CE0B695A79597958795FC
:1037D0002A95D1F7807F2D813E819F819F70892B13
:1037E0008583368327834114510409F04BC0A80117
:1037F00068E08AE10E942917209248073092490721
:1038000060924A0770924B0780924C0790924D0746
:10381000FD85F0934E078E8580934F07C8012E9645
:103820000FB6F894DEBF0FBECDBFDF91CF911F91D1
:103830000F91FF90EF90DF90CF90BF90AF909F904F
:103840008F907F906F905F904F903F902F900C944F
:10385000FB2CE0915A07F0915B07EE0FFF1FEE0F74
:10386000FF1FEC59F84FA080B180C280D380FE01C9
:1038700031967F0181019A01AB016D857E8581E0E2
:1038800090E08CCF4A94452849F6A80168E082E28E
:103890000E942917209250073092510760925207D8
:1038A000709253078092540790925507ED85E093EC
:1038B0005607FE85F0935707B1CF2F923F924F9254
:1038C0005F926F927F928F929F92AF92BF92CF92B0
:1038D000DF92EF92FF920F931F93CF93DF93CDB7B9
:1038E000DEB7E5970FB6F894DEBF0FBECDBFE22E70
:1038F00029A3F32E3AA34BA35CA36DA37EA38FA3AE
:1039000098A7702E612E9701AFEF0E94472C2E379B
:103910003A4146405105610571058105910509F05F
:1039200058F480E889A38AE18AA386E08BA31CA2CD
:103930001DA21EA21FA218A629A13AA14BA15CA1FB
:103940006DA17EA18FA198A52115314C4A415D43FF
:10395000654071058105910569F060F019A281EC5F
:103960008AA38AE18BA38DE38CA385E08DA31EA29D
:103970001FA218A6D9A04AA05BA0ACA0EDA0FEA0F3
:103980000FA118A5272C362C2D2D342D452D5A2D61
:10399000B701C8012115344E4B40544562407105B2
:1039A0008105910509F008F425C1A8E04A2EA7E099
:1039B0005A2E2FEE36E03AA729A78901F201D12C21
:1039C000C101880F991FDC01A850B94F7D012081EA
:1039D00031814281538164817581868197813896D6
:1039E0002115344E4B4054456240710581059105C7
:1039F00071F068F0D71459F0D80119962D913C91C7
:103A0000D7018D919C912817390709F46AC1D39485
:103A10000E5F1F4FB6E0DB12DACF81010259184F5B
:103A2000F8018081811108C061E0872D962D0E94E8
:103A3000DF1981E0D8018C9329A13AA14BA15CA1A7
:103A40006DA17EA18FA198A5D101E3E0AA0FBB1FB4
:103A5000EA95E1F7A151B94FFD01799659962C935A
:103A60003183428353836483758386839783FE0106
:103A70003D964F01A12CB12CC12CD12CE12CF12C65
:103A800000E010E00E946B082BA73CA74DA75EA7A3
:103A90006FA778AB89AB9AABC101880F991F9C01C6
:103AA0002151394F7901D90119960D911C912BA5FE
:103AB0003CA589A99AA90E94931B712C612CF7013E
:103AC0003996FDABECABD201AC901196EC9011970E
:103AD0001296FC90129713960C91139714961C91C2
:103AE00014971596BC91F201D680C780F8E04F0E6E
:103AF000511C2A2D3E2D4F2D502F612F7B2F8D2DA8
:103B00009C2DA0E00E94532C09F455C0E9A5FAA50C
:103B100021853285ECA9FDA980819181281739077B
:103B200009F049C0A98EEA8EFB8E0C8F1D8FBE8FC7
:103B3000DF8EC8A2CE0149960E94810A8BAB298DE7
:103B40003A8D4B8D5C8D6D8D7E8DCE0101964C0135
:103B5000ABA4BCA4CDA4DEA4EFA4F8A809A91AA91B
:103B60008F8D98A10E946B08AA24A394298D3A8D69
:103B70004B8D5C8D6D8D7E8D8F8D98A12F3F354D3A
:103B800041415E47634071058105910509F008F4E4
:103B9000A12CAF928BA8C980DA80EB80FC800D81CC
:103BA0001E812F81388549855A856B857C85C301A7
:103BB0000E94A81A0F90BFEF6B1A7B0AE9A5FAA51D
:103BC0003296FAA7E9A7F6E06F16710409F07BCFE9
:103BD000F101EE0FFF1FE151F94F8185928560E2FF
:103BE000009719F0019721F460E881EB0E940F170C
:103BF00080E078C0D10193E0AA0FBB1F9A95E1F74E
:103C0000A151B94FFD0179965996DC9241825282B9
:103C1000A382E482F5820683178381010259184F3B
:103C2000D8018C91811108C061E0872D962D0E94EA
:103C3000DF1981E0F8018083CE0181960E94810A1C
:103C4000582EF101EE0FFF1FE151F94F0184F2856B
:103C5000E02D29A13AA14BA15CA16DA17EA18FA16C
:103C600098A5EF2B51F5A0904807B0904907C09058
:103C70004A07D0904B07E0904C07F0904D07009119
:103C80004E0710914F07DE011D964D010E946B08F3
:103C90001F92852CA12CCD84DE84EF84F8880989BD
:103CA0001A892B893C894D895E896F89788D872D8A
:103CB000962D0E94A81A0F909BCFA0905007B0900D
:103CC0005107C0905207D0905307E0905407F090EE
:103CD00055070091560710915707FE013D964F0179
:103CE000D5CF81E0E5960FB6F894DEBF0FBECDBF0D
:103CF000DF91CF911F910F91FF90EF90DF90CF90C8
:103D0000BF90AF909F908F907F906F905F904F90FB
:103D10003F902F9008952F923F924F925F926F9213
:103D20007F928F929F92AF92BF92CF92DF92EF924B
:103D3000FF920F931F9360915E0670915F068091D2
:103D400060069091610628EE33E040E050E00E946A
:103D5000F72AC0906A06D0906B06E0906C06F0904F
:103D60006D0656016701E12CF12C00E010E00E9485
:103D70003E2CE4E6AE2EB12CC12CD12C0E949F2A01
:103D800010E000E00E945D1C01E010E020E430EB58
:103D90004EE45AE260E070E080E090E00E945D1C3A
:103DA00002E010E020EC3AEC44E55AE260E070E01A
:103DB00080E090E00E945D1C1F910F91FF90EF90BA
:103DC000DF90CF90BF90AF909F908F907F906F903B
:103DD0005F904F903F902F9008950F931F936093A3
:103DE0006407709365078093660790936707E8E41C
:103DF000F7E020813181428153816481758110E037
:103E000000E0868197810E94931BE0E5F7E0208126
:103E10003181428153816481758101E010E08681A6
:103E200097810E94931B1F910F9108958F929F92EB
:103E3000AF92BF920F931F93CF93DF93CDB7DEB7AF
:103E4000A1970FB6F894DEBF0FBECDBF19A24230C6
:103E500008F44AE08E010F5D1F4F842E912CB12C87
:103E6000A12CA50194010E94682AE62FB901CA017C
:103E7000EA3044F5E05DD801EE938D01232B242B2D
:103E8000252B79F790E080E0109769F0FD01019013
:103E90000020E9F73197AF014A1B5B0BBD0186E7B4
:103EA00097E00E94EE0BA1960FB6F894DEBF0FBE0E
:103EB000CDBFDF91CF911F910F91BF90AF909F9099
:103EC0008F900895E95CD7CFFC0101900020E9F7BD
:103ED0003197AF01481B590BBC0186E797E00C9462
:103EE000EE0B0E94842D1F920F920FB60F92112499
:103EF0002F933F938F939F93AF93BF9380915006DF
:103F000090915106A0915206B091530630914F0600
:103F100023E0230F2D3758F50196A11DB11D2093E5
:103F20004F068093500690935106A0935206B0938B
:103F300053068091540690915506A0915606B09173
:103F400057060196A11DB11D809354069093550606
:103F5000A0935606B0935706BF91AF919F918F9152
:103F60003F912F910F900FBE0F901F90189526E84C
:103F7000230F0296A11DB11DD2CF1F920F920FB633
:103F80000F9211242F933F934F935F936F937F93DF
:103F90008F939F93AF93BF93EF93FF938091B9005B
:103FA000887F803609F44AC0F0F5883209F4A7C04A
:103FB00018F5803109F49BC0B8F4882309F4F9C0DE
:103FC000883009F494C0FF91EF91BF91AF919F9118
:103FD0008F917F916F915F914F913F912F910F90B2
:103FE0000FBE0F901F901895883109F488C0803259
:103FF00051F78093BC0614C0803409F49DC040F48E
:104000008033B9F38833F9F68093BC0685ECB0C0F1
:10401000803509F485C0883509F496C0883499F64E
:104020000E946016D0CF883909F48CC038F58837E3
:1040300029F050F4883611F0803729F683E0809318
:10404000BE0610924E0657C0883809F47BC08039EE
:1040500019F0803809F0B7CF80914E06803208F011
:1040600071C0E0914E0681E08E0F80934E068091E4
:10407000BB00F0E0E25DF94F80833DC0803B39F04A
:10408000E0F4803A09F479C0883A09F09CCF84E0E2
:104090008093BE0610922D0610922C06E0917406B5
:1040A000F0917506099580912C0681110FC081E071
:1040B00080932C0610920C0609C0803C09F4A6CF10
:1040C000883C09F4A3CF883B09F07DCFE0912D0611
:1040D00081E08E0F80932D06F0E0E45FF94F808140
:1040E0008093BB0090912D0680912C0629C0809171
:1040F00099068093BB0085EC8093BC0064CF9091BF
:10410000BB068091BA06981758F5E091BB0681E08E
:104110008E0F8093BB06F0E0E656F94F8081E9CF21
:10412000E091BB0681E08E0F8093BB068091BB00BF
:10413000F0E0E656F94F80839091BB068091BA0675
:104140009817C8F285E8D8CFE091BB0681E08E0FC2
:104150008093BB068091BB00F0E0E656F94F808368
:104160008091BD0681115CCF81E08093980684EA3E
:104170008093BC001092BE0626CF85EC8093BC00D5
:104180001092BE0680914E06803230F4E0914E06C9
:10419000F0E0E25DF94F108260914E0670E0E09130
:1041A0007206F09173068EE296E0099510924E0623
:1041B0000ACF1092BC0634CF1F920F920FB60F9207
:1041C00011242F933F934F935F936F937F938F931C
:1041D0009F93AF93BF93CF93DF93EF93FF93809120
:1041E000A7070E94440CEC018091A6070E94440C92
:1041F0009091A5079F70CC0FDD1FC82B24E0929FE4
:10420000C0011124895F9A4FC80FD92FD11D888111
:104210008093A50780738031B9F481E090E00E941B
:10422000B118FF91EF91DF91CF91BF91AF919F9125
:104230008F917F916F915F914F913F912F910F904F
:104240000FBE0F901F901895803259F78FEF9FEF98
:10425000E6CFCF93DF93E3EEF6E01382128288EE8F
:1042600093E0A0E0B0E084839583A683B7838BE3DB
:1042700095E091838083C5EAD7E082E0898383E07B
:104280008A8360E082E00E94CD0C60E08A810E9417
:10429000CD0C61E089810E946D0C61E08A810E94F1
:1042A0006D0C1882E6E7F7E01382128220E830E016
:1042B0003583248380E490E0978386833187208749
:1042C00093878287168A158614861786168681E05C
:1042D000858B848B2FEF3FEF338B228B318B208BA1
:1042E000878B108E128E118E8DE495E091838083E2
:1042F0008FEF858F81A3878F868F84E080A3EFEE79
:10430000F6E085E0DF011D928A95E9F715821682B5
:104310001782108680E680936D0780E498E7ADE70A
:10432000B1E080935C0790935D07A0935E07B09324
:104330005F07109259071092580710925B0710926E
:104340005A0710926C07DF91CF910895CF93DF93B6
:10435000CDB7DEB766970FB6F894DEBF0FBECDBF00
:10436000789484B5826084BD84B5816084BD85B550
:10437000826085BD85B5816085BD80916E0081605C
:1043800080936E0010928100809181008260809302
:104390008100809181008160809381008091800004
:1043A0008160809380008091B10084608093B1002F
:1043B0008091B00081608093B00080917A00846029
:1043C00080937A0080917A00826080937A00809155
:1043D0007A00816080937A0080917A00806880936F
:1043E0007A001092C1000E949B0C82E08093920799
:1043F0008CE380939107809193078F3F09F48CC6DB
:1044000061E0809195070E94CD0C61E08091970753
:104410000E94CD0C80919707082E000C990BFC018F
:10442000E255FA4FE491F0E0EE0FFF1FEC55FA4F22
:104430002591349130939E0720939D07FC01E0570E
:10444000FA4FE491E093A30780919507082E000CA2
:10445000990BFC01E255FA4FE491F0E0EE0FFF1FDB
:10446000EC55FA4F259134913093A00720939F0784
:10447000FC01E057FA4FE491E093A407809198077C
:1044800081113EC061E0809193070E94CD0C61E0F4
:10449000809194070E94CD0C80919407082E000C07
:1044A000990BFC01E255FA4FE491F0E0EE0FFF1F8B
:1044B000EC55FA4F2591349130939C0720939B073C
:1044C000FC01E057FA4FE491E093A2078091930733
:1044D000082E000C990BFC01E255FA4FE491F0E034
:1044E000EE0FFF1FEC55FA4F2591349130939A0748
:1044F00020939907FC01E057FA4FE491E093A1075C
:1045000080919807882309F439C01FB7F8948091E7
:104510005806811127C0E8EBF5E08491EAE9F5E05F
:104520009491E82FF0E0EE0FFF1FEA57FA4FA591A4
:10453000B491EC91E92321F461E08AE00E946D0CD2
:1045400061E08AE00E94CD0C8CB580618CBD8CB599
:1045500080648CBD61E08DE00E94CD0C61E08BE059
:104560000E94CD0C809158068F5F809358061FBF24
:104570008CB58C7F8CBD8DB581608DBD61E08091E7
:1045800096070E94CD0C61E0809196070E946D0C09
:1045900061E070E080E090E00E942E0D60E080918C
:1045A00096070E946D0C6AE070E080E090E00E9447
:1045B0002E0D61E0809196070E946D0C8EEA0E949C
:1045C000571785ED0E94571780E80E94571788EA11
:1045D0000E9457178FE30E94571783ED0E945717C9
:1045E00080E00E94571780E40E9457178DE80E94D0
:1045F000571784E10E94571780E20E94571780E006
:104600000E94571781EA0E94571788EC0E9457179B
:104610008AED0E94571782E10E94571781E80E9495
:1046200057178FEC0E94571789ED0E94571781EF9B
:104630000E9457178BED0E94571780E40E9457176E
:1046400084EA0E94571786EA0E9457178FEA0E9451
:104650005717E1E0F1E080E094E0DF019C011D925A
:1046600021503040E1F781E090E0909389078093FA
:10467000880790938707809386070E94AB1762E0B4
:1046800082E00E94CD0C62E083E00E94CD0C62E0EB
:1046900086E00E94CD0C62E08EE00E94CD0C62E0CC
:1046A0008FE00E94CD0C62E080E10E94CD0C62E0C0
:1046B00084E10E94CD0C0E949B0C80916D0791E0DB
:1046C0009093BF068093E1061092C0061092E20616
:1046D0000E940C0381110BC180E00E944B1990E0F5
:1046E000880F892F881F990B0197B1F362E987EB37
:1046F0000E940F1780E498E7ADE7B1E080935C0774
:1047000090935D07A0935E07B0935F0760E070E051
:10471000CB010E94ED1E60E880E10E940F1760E867
:1047200081E10E940F1760E882E10E940F1760E8A4
:1047300083E10E940F1760E884E10E940F1760E890
:1047400085E10E940F1760E886E10E940F1760E87C
:1047500087E10E940F176CE080E10E940F176CE068
:1047600081E10E940F176CE082E10E940F176CE05C
:1047700083E10E940F176CE084E10E940F176CE048
:1047800085E10E940F176CE086E10E940F176CE034
:1047900087E10E940F1710E000E020E030E24FE5D3
:1047A00050EA62E170E080E090E00E94931B01E03B
:1047B00010E020E030E24FE550EA62E170E080E096
:1047C00090E00E94931B1092F9061092F806109246
:1047D000FB061092FA061092FD061092FC0610924B
:1047E000FF061092FE061092010710920007109229
:1047F00003071092020781E090E0909305078093F1
:104800000407909307078093060770E060E090E04C
:1048100080E00E94F71970E060E081E090E00E9483
:10482000F71970E060E082E090E00E94F71970E014
:1048300060E083E090E00E94F71970E060E084E0BF
:1048400090E00E94F71970E060E085E090E00E943F
:10485000F71961E070E086E090E00E94F71961E0EE
:1048600070E087E090E00E94F71960E082EA0E9421
:104870000F1760E083EA0E940F1760E084EA0E944D
:104880000F1760E281EB0E940F1760E881EB0E9436
:104890000F1708E017E05EE6C52E57E0D52EF12C85
:1048A000E12CD8011C9211961C92119712961C9221
:1048B000129713961C92139714961C9214971596A0
:1048C0001C92159716961C92169717961C92085FC5
:1048D0001F4F60E0C7010E94DF19F60111926F01BE
:1048E000FFEFEF1AFF0A28E0E216F104D1F668E4C0
:1048F00078EE81E090E00E94ED1E80E10E944B196D
:10490000682F636080E10E940F1781E10E944B19BC
:10491000682F6C7F81E10E940F1782E10E944B1982
:10492000682F6C7F82E10E940F1761E090E080E0C9
:104930000E94DF1964E181E090E00E94DF1961E0EC
:1049400082E090E00E94DF1980916800846080938B
:10495000680080916D008C6080936D00789412E007
:10496000109359060E941A1A10935A060E947C1836
:1049700048EE442E43E0542E612C712CCE01039658
:10498000998B888BCC24C394D12C37E1232E312CE6
:1049900080906A0690906B06A0906C06B0906D06B1
:1049A00080916E0690916F06A0917006B09171068D
:1049B00088159905AA05BB05A1F00E94600D6093BA
:1049C00066067093670680936806909369060E9456
:1049D0008B1E80926E0690926F06A0927006B09227
:1049E000710680905E0690905F06A0906006B09081
:1049F00061068091620690916306A0916406B09171
:104A0000650688159905AA05BB05A1F00E94600DF1
:104A100060936606709367068093680690936906B4
:104A20000E948B1E8092620690926306A09264069A
:104A3000B092650610915C0680915D06811761F069
:104A40000E94600D60936606709367068093680607
:104A50009093690610935D068EE00E94440C892BAA
:104A6000B1F40E94600D645D7E4F8F4F9F4F609345
:104A700066067093670680936806909369060E94A5
:104A80007C186CE271E080E090E00E942E0D8FE0D7
:104A90000E94440C892B21F50E94600D645D7E4FBD
:104AA0008F4F9F4F609366067093670680936806EA
:104AB00090936906809159068F5F863008F02FC366
:104AC000809359060E941A1A62E370E080E090E039
:104AD0000E942E0D6CE271E080E090E00E942E0DAD
:104AE00080E10E94440C892B09F01BC30E94600DD9
:104AF000645D7E4F8F4F9F4F60936606709367068D
:104B0000809368069093690681E080935B0684E158
:104B10000E94440C892B09F007C30E94600D645D5C
:104B20007E4F8F4F9F4F609366067093670680930A
:104B300068069093690681E080935B068090660624
:104B400090906706A0906806B090690694E6890E7A
:104B5000911CA11CB11C0E94600D681579058A0585
:104B60009B0508F057C480906A0690906B06A09051
:104B70006C06B0906D06C501B40120E432E44FE04C
:104B800050E00E94682AF22EE32E022F132FA30179
:104B900092010E94682A2A8B3E8BC501B401A301B1
:104BA00092010E94682AA1E0B1E0E0E0F4E01D92E9
:104BB0003197E9F722E020938A0720938B071A8226
:104BC00019822DE0A889B9891D922A95E9F7011566
:104BD000110509F0ACC289E290E0909383078093BD
:104BE0008207D0928507C09284077F936F93BE8916
:104BF000BF93EA89EF9389E795E09F938F9321E034
:104C000030E02C0F3D1F3F932F930E94892D0FB64C
:104C1000F894DEBF0FBECDBFCE0101960E94641F87
:104C2000D0928907C0928807D0928707C0928607E2
:104C3000EE24E394F12C04E110E02FE730E044E1AE
:104C400050E070E060E086E797E00E9436140BE2E7
:104C500010E02FE730E04BE250E070E060E086E7E4
:104C600097E00E94361407E210E029E630E048E1C0
:104C700050E069E670E086E797E00E94361427E589
:104C800030E048E150E067E570E086E797E00E9499
:104C900036140FE310E027E530E040E350E067E52D
:104CA00070E086E797E00E94361407E310E022E503
:104CB00030E047E350E06FE070E086E797E00E9465
:104CC000361481E080938A0780938B072BE330E0D2
:104CD00030938307209382073092850720928407C0
:104CE00084E995E00E94641F86E390E09093830737
:104CF0008093820781E290E09093850780938407F8
:104D000080915A06823021F489E995E00E94641F5F
:104D100080915A06833021F48FE995E00E94641F48
:104D200080915A06843021F484EA95E00E94641F41
:104D300080915A06853021F48AEA95E00E94641F2A
:104D400080915A06863021F480EB95E00E94641F22
:104D500080915A06813021F48AEA95E00E94641F0E
:104D600081E080938A0780938B070CE510E0109315
:104D700083070093820780E390E0909385078093F8
:104D8000840785EB95E00E94641F109383070093CE
:104D9000820789E390E09093850780938407809051
:104DA0005E0690905F06A0906006B09061064AE0B3
:104DB000C501B401B7FE0DC06DE286E797E00E9421
:104DC000051366277727CB01681979098A099B099A
:104DD0004AE00E94161F89EB95E00E94641F81E063
:104DE00080938A0780938B078EE690E090938307E9
:104DF00080938207309285072092840780916A060B
:104E000090916B06A0916C06B0916D06803492442F
:104E1000AF40B10520F486EA95E00E94641F8091BE
:104E20006A0690916B06A0916C06B0916D06803475
:104E30009244AF40B10520F08BEB95E00E94641FD7
:104E40008EE690E0909383078093820781E290E062
:104E5000909385078093840780915E0690915F060A
:104E6000A0916006B0916106892B8A2B8B2B21F4CF
:104E70008FEB95E00E94641F80915E0690915F0623
:104E8000A0916006B0916106892B8A2B8B2B21F0B3
:104E900083EC95E00E94641F8BE590E0909383077C
:104EA000809382078CE190E090938507809384073C
:104EB00080915B06811104C087EC95E00E94641F1D
:104EC00080915B068111D5C210925E0610925F063A
:104ED000109260061092610680915B06882341F073
:104EE00010925E0610925F061092600610926106A4
:104EF00082E080938A0780938B0710928307109239
:104F0000820789E190E090938507809384078091E0
:104F10005906813021F48AEC95E00E94641F80914B
:104F20005906823021F48EEC95E00E94641F809136
:104F30005906833021F482ED95E00E94641F809130
:104F40005906843021F486ED95E00E94641F80911B
:104F50005906853021F483EE95E00E94641F80910C
:104F60005906863021F483EE95E00E94641F8091FB
:104F70005906873021F48EEC95E00E94641F8091E1
:104F80005906883021F48AED95E00E94641F8091D3
:104F90005906893021F48EED95E00E94641F8091BE
:104FA00059068A3021F482EE95E00E94641F8091B8
:104FB00059068B3021F482ED95E00E94641F8091A8
:104FC00059068C3021F486EE95E00E94641F809192
:104FD00059068D3021F48AEE95E00E94641F80917D
:104FE00059068E3021F48EEE95E00E94641F809168
:104FF00059068F3021F482EF95E00E94641F809162
:105000005906803121F486ED95E00E94641F80915D
:105010005906813121F48BEE95E00E94641F809146
:105020005906823121F486EF95E00E94641F809139
:105030005906833121F48AEF95E00E94641F809124
:105040005906843121F483EE95E00E94641F80911B
:105050005906853121F483EF95E00E94641F809109
:105060005906813009F0A8C010925E0610925F06C2
:1050700010926006109261062091000130E050E02D
:1050800040E02150310941095109ADE0B0E00E94F2
:105090005D2A29E230E040E050E00E943E2ADA0139
:1050A000C9010196A11DB11D8A8B9B8BAC8BBD8B59
:1050B00081E080938A0780938B0710928307109278
:1050C000820780E390E090938507809384078EEFBA
:1050D00095E00E94641FEA89E150EE3008F078C044
:1050E000F0E0E258F74DEE24E394F12C06E010E0F6
:1050F00022E030E040E350E00C94992AE2280F29A6
:105100001229152918291B291E2921292429272973
:105110002A292D29302933290E949B0C2FCA81E08E
:10512000CFCC10925B06F3CC10925B0607CD043611
:105130001105F8F485E090E090938307809382074F
:10514000D0928507C09284077F936F939E899F9327
:10515000AA89AF93EF92FF9285E795E09F938F9393
:10516000E1E0F0E0EC0FFD1FFF93EF930E94892D2B
:105170004ECD25E030E03093830720938207D09214
:105180008507C09284072AE030E040E050E00E94AA
:10519000682A3F932F933E893F938A898F93EF929A
:1051A000FF9285E895E09F938F93A1E0B0E0AC0F6C
:1051B000BD1FBF93AF93DACF80915B06882309F4BC
:1051C00053CF5ACF6FE070E086E797E00E94CB1490
:1051D000109283071092820789E390E090938507ED
:1051E0008093840781E096E00E94641FE0915C0652
:1051F000E150EE3008F00CC1F0E0EF5FF64D0C949A
:10520000992AF929EA29DB29CC29BD29AE299F2928
:10521000902981297229632954294529362964E175
:1052200070E0D2CF69E170E0CFCF6EE170E0CCCF1B
:1052300063E270E0C9CF68E270E0C6CF6DE270E073
:10524000C3CF62E370E0C0CF67E370E0BDCF6CE333
:1052500070E0BACF61E470E0B7CF66E470E0B4CF3D
:105260006BE470E0B1CF60E570E0AECFEE24E39484
:10527000F12C06E010E022E030E04AE350E060E587
:1052800070E086E797E00E94CB14EE24E394F12CC3
:1052900006E010E022E030E04AE350E06BE470E02A
:1052A00086E797E00E94CB14EE24E394F12C06E00D
:1052B00010E022E030E04AE350E066E470E086E788
:1052C00097E00E94CB14EE24E394F12C06E010E06A
:1052D00022E030E04AE350E061E470E086E797E0E6
:1052E0000E94CB14EE24E394F12C06E010E022E0BF
:1052F00030E04AE350E06CE370E086E797E00E941C
:10530000CB14EE24E394F12C06E010E022E030E030
:105310004AE350E067E370E086E797E00E94CB1431
:10532000EE24E394F12C06E010E022E030E04AE3C2
:1053300050E062E370E086E797E00E94CB14EE2431
:10534000E394F12C06E010E022E030E04AE350E084
:105350006DE270E086E797E00E94CB14EE24E394C0
:10536000F12C06E010E022E030E04AE350E068E291
:1053700070E086E797E00E94CB14EE24E394F12CD2
:1053800006E010E022E030E04AE350E063E270E043
:1053900086E797E00E94CB14EE24E394F12C06E01C
:1053A00010E022E030E04AE350E06EE170E086E792
:1053B00097E00E94CB14EE24E394F12C06E010E079
:1053C00022E030E04AE350E069E170E086E797E0F0
:1053D0000E94CB14EE24E394F12C06E010E022E0CE
:1053E00030E04AE350E064E170E086E797E00E9435
:1053F000CB14EE24E394F12C06E010E022E030E040
:105400004AE350E06FE070E086E797E00E94CB143B
:105410000E94AB1783E480937C0080917A008064C3
:1054200080937A0080917A0086FDFCCF809178008D
:1054300020917900322F282FADE0B0E00E948A2A17
:105440002FE231E040E050E00E943E2ADA01C9013B
:105450000196A11DB11D8F3050F480935C0680E051
:1054600090E0892B09F494CA0E9400008BCA8EE058
:10547000F4CF84E096E00E94641F2ECD052E97FBAA
:105480001EF400940E94552A57FD07D00E94682AF6
:1054900007FC03D04EF40C94552A50954095309556
:1054A00021953F4F4F4F5F4F089590958095709590
:1054B00061957F4F8F4F9F4F08950E948A2AA59F25
:1054C000900DB49F900DA49F800D911D11240895FF
:1054D000A1E21A2EAA1BBB1BFD010DC0AA1FBB1FF8
:1054E000EE1FFF1FA217B307E407F50720F0A21B6A
:1054F000B30BE40BF50B661F771F881F991F1A94D7
:1055000069F760957095809590959B01AC01BD0100
:10551000CF010895A29FB001B39FC001A39F700D5A
:10552000811D1124911DB29F700D811D1124911DAB
:105530000895EE0FFF1F0590F491E02D0994DF937D
:10554000CF931F930F939A9DF02D219FF00D8B9D6C
:10555000F00D8A9DE02DF10D039FF00D029FE00DEF
:10556000F11D4E9DE00DF11D5E9DF00D4F9DF00D66
:105570007F936F93BF92AF925F934F93D5010E9439
:105580008A2A8B01AC01D7010E948A2AEB01E80F1D
:10559000F91FD6010E94EE2A2F913F91D6010E9459
:1055A0008A2AC60FD71FE81FF91FAF91BF910E942B
:1055B000EE2A2F913F910E948A2AC60FD71FE81F1B
:1055C000F91FD6010E948A2AE60FF71F9801BE0133
:1055D000CF010F911F91CF91DF9108950E948A2AE8
:1055E000460F571FC81FD91F08F43196089597FB1F
:1055F00057FF0C94072B9F938F930E94072B6E1BD2
:105600007F0BAF91BF918A0B9B0B0895E894DF93BA
:10561000CF93FC01DB010E948A2A7F936F93E901FB
:105620009A01AC01BF93AF933F932F93DF010E9488
:105630008A2A26F46C1B7D0B820B930B9E01EB01D7
:10564000FC010E94EE2AAF91BF912F913F910E94E1
:10565000EE2ABE01CF01F9012F913F91CF91DF9149
:105660000895689401C0E894F92FF12B12F00C947E
:10567000652BA0E0B0E0EFE3FBE20C94D72B092E02
:10568000059422F40E94C12B112392F4F0E80F2616
:10569000FFEFE094F09400951095B094C094D094EE
:1056A000A194BF0ACF0ADF0AEF0AFF0A0F0B1F0BF4
:1056B0000E94702B07FC0E94C12BCDB7DEB7ECE037
:1056C0000C94F32B689401C0E8948F929F92CF932F
:1056D000DF930E94702BDF91CF919F908F90089560
:1056E00088249924F401E401B0E49F93AA279A1531
:1056F0008B049C04ED05FE05CF05D007A10798F4A7
:10570000AD2FDC2FCF2FFE2FE92D982C892E982F2F
:10571000872F762F652F542F432F322F2227B850F3
:1057200031F7BF9127C01B2EBF91BB27220F331F1C
:10573000441F551F661F771F881F991F881C991CBF
:10574000EE1FFF1FCC1FDD1FAA1FBB1F8A149B0467
:10575000EC05FD05CE05DF05A007B10748F08A1866
:105760009B08EC09FD09CE09DF09A00BB10B2160F4
:105770001A94E1F62EF49401AF01BE01CD01000CA4
:1057800008956095709580959095309540955095C9
:1057900021953F4F4F4F5F4F6F4F7F4F8F4F9F4F21
:1057A00008952F923F924F925F926F927F928F92C5
:1057B0009F92AF92BF92CF92DF92EF92FF920F93A0
:1057C0001F93CF93DF93CDB7DEB7CA1BDB0B0FB6AA
:1057D000F894DEBF0FBECDBF09942A883988488867
:1057E0005F846E847D848C849B84AA84B984C884FD
:1057F000DF80EE80FD800C811B81AA81B981CE0FF4
:10580000D11D0FB6F894DEBF0FBECDBFED010895D8
:10581000002E083090F0982F872F762F652F542F69
:10582000432F322F22270850F4CF220F331F441F5B
:10583000551F661F771F881F991F0A95B2F7002D05
:10584000089597FD1094002E083098F00850232FEB
:10585000342F452F562F672F782F892F912DF4CF76
:1058600015949795879577956795579547953795AB
:1058700027950A95AAF71124002D08952A0D3B1D9E
:105880004C1D5D1D6E1D7F1D801F911F08950024FE
:10589000A7FD00942A0F301D401D501D601D701D76
:1058A000801D901D08950024A7FD00942A1730053F
:1058B00040055005600570058005900508950F931B
:1058C0001F93CF93DF938230910510F482E090E034
:1058D000E091AA07F091AB0730E020E0B0E0A0E053
:1058E000309799F42115310509F44AC0281B390B6A
:1058F00024303105D8F58A819B816115710589F1C4
:10590000FB0193838283FE0111C04081518102819A
:10591000138148175907E0F04817590799F4109771
:1059200061F012960C93129713961C933296CF0146
:10593000DF91CF911F910F9108950093AA071093C3
:10594000AB07F4CF2115310551F04217530738F05A
:10595000A901DB019A01BD01DF01F801C1CFEF010F
:10596000F9CF9093AB078093AA07CDCFFE01E20F4A
:10597000F31F819391932250310939832883D7CF24
:105980002091A8073091A907232B41F4209103050A
:10599000309104053093A9072093A80720910105B1
:1059A000309102052115310541F42DB73EB74091E4
:1059B000050550910605241B350BE091A807F091D1
:1059C000A907E217F307A0F42E1B3F0B281739078E
:1059D00078F0AC014E5F5F4F2417350748F04E0F4B
:1059E0005F1F5093A9074093A807819391939FCF7E
:1059F000F0E0E0E09CCFCF93DF930097E9F0FC016B
:105A0000329713821282A091AA07B091AB07ED01E1
:105A100030E020E01097A1F420813181820F931FA4
:105A20002091A8073091A9072817390709F061C00C
:105A3000F093A907E093A807DF91CF910895EA01B9
:105A4000CE17DF07E8F54A815B819E0141155105BC
:105A5000B1F7E901FB83EA8349915991C40FD51F3E
:105A6000EC17FD0761F4808191810296840F951FE8
:105A7000E90199838883828193819B838A83F0E003
:105A8000E0E012968D919C9113970097B9F52D91B6
:105A90003C911197CD010296820F931F2091A80788
:105AA0003091A9072817390739F6309751F5109228
:105AB000AB071092AA07B093A907A093A807BCCF81
:105AC000D383C28340815181840F951FC817D907A2
:105AD00061F44E5F5F4F88819981480F591F518350
:105AE00040838A819B81938382832115310509F04C
:105AF000B0CFF093AB07E093AA079ECFFD01DC0186
:105B0000C0CF13821282D7CF81E090E0F8940C943A
:105B10002A30AEE0B0E0EFE8FDE20C94DF2B0D8917
:105B20001E8986E08C831A8309838FEF9FE79E830B
:105B30008D83AE01475E5F4F6F89788DCE010196F0
:105B40000E94AC2D2F813885020F131FF80110829F
:105B50002E96E4E00C94FB2BABE0B0E0E2EBFDE230
:105B60000C94D12B7C013B018A01FC011782168227
:105B7000838181FFC8C1CE0101965C01F701938149
:105B8000F30193FD859193FF81913F01882309F4EF
:105B900053C1853239F493FD859193FF81913F0183
:105BA000853229F4B70190E00E949C2FE7CF912C19
:105BB000212C312CFFE1F31538F08B3211F190F4E8
:105BC000803209F1833229F137FC3CC020ED280FE7
:105BD0002A3050F536FE20C08AE0989E200D112410
:105BE000922E06C08D3291F0803371F7689430F8B0
:105BF000F30193FD859193FF81913F018111DACFEC
:105C000021C0689431F8689432F8F2CF689433F880
:105C1000EFCF689434F8ECCFEAE02E9E200D1124EB
:105C2000222E689435F8E4CF8E3229F436FC04C174
:105C3000689436F8DDCF8C3619F4689437F8D8CFED
:105C40008836B1F2982F9F7D95549330E0F08336DB
:105C5000A1F18337C1F1833509F063C02801F2E077
:105C60004F0E511CF801C080D180692D70E036FCC8
:105C700002C06FEF7FEFC6010E94862F4C0168942F
:105C800037F882010AC00C5F1F4FFFE3F9838824B5
:105C90008394912C6501E89437F833FE2DC0522C83
:105CA0008114910471F5552009F468CFB70180E2A1
:105CB00090E00E949C2F5A94F6CFF801808189834E
:105CC0000E5F1F4FE4CF2801F2E04F0E511CF80188
:105CD000C080D180692D70E036FC02C06FEF7FEF8D
:105CE000C6010E94912F4C018201D5CFB70180E2FD
:105CF00090E00E949C2F2A942814190409F0B0F710
:105D0000CECFF60137FC859137FE81916F01B70147
:105D100090E00E949C2F51105A94F1E08F1A910844
:105D2000BFCF843619F0893609F077C0F80137FE05
:105D30006BC060817181828193810C5F1F4FF32D55
:105D4000FF763F2E97FF09C09095809570956195DD
:105D50007F4F8F4F9F4F689437F82AE030E0A501BE
:105D60000E94CC2FC82ECA188C2C432C36FE0CC097
:105D7000E89440F8C91440F434FE05C032FC03C076
:105D8000F32DFE7E4F2E892C44FE95C0FE01EC0DB6
:105D9000F11D8081803309F087C0242D297E422E99
:105DA000842D8870582E43FC95C040FE8FC09C2CDB
:105DB000821418F42C0C922C981844FE91C0B70150
:105DC00080E390E00E949C2F42FE09C088E790E0AB
:105DD00041FE02C088E590E0B7010E949C2FC914E3
:105DE00008F48AC0CA94D12C9FEFC91AD90ACA0CE8
:105DF000DB1CF60182916F01B70190E00E949C2F9D
:105E0000AC14BD04B1F74FCF60817181072E000C37
:105E1000880B990B0E5F1F4F92CFD32CE894D4F8C8
:105E20002AE030E0853739F1232D297FD22E8F36B5
:105E300001F148F48835A9F0F701868197812B9606
:105E4000E2E10C94ED2B803749F08837A9F7D4FEB6
:105E500002C06894D2F820E130E00DC06894D4F814
:105E6000F6CF34FE03C0822F8660D82E20E132E0C8
:105E700002C028E030E0F801D7FE0FC060817181D8
:105E8000828193810C5F1F4FA5010E94CC2FC82EE9
:105E9000CA183D2CE89437F867CF6081718190E093
:105EA00080E00E5F1F4FF0CF42FC02C0839478CF9A
:105EB0008394839475CF842D867809F471CFF6CFBF
:105EC000B70180E290E00E949C2F83948214C0F37B
:105ED000512C73CF522C5818821408F46ECFF8CF7F
:105EE000842D867809F47BCF8BE241FE80E247FC6B
:105EF0008DE2B70190E071CFB70180E390E00E949E
:105F00009C2F9A946CCF8FEF9FEF99CFFC01059057
:105F1000615070400110D8F7809590958E0F9F1FAB
:105F20000895FC016150704001900110D8F78095F0
:105F300090958E0F9F1F08950F931F93CF93DF931C
:105F4000182F092FEB018B8181FD09C01FEF0FEF87
:105F5000812F902FDF91CF911F910F91089582FF94
:105F600014C02E813F818C819D81281739073CF414
:105F7000E881F981CF0101969983888310838E810E
:105F80009F8101969F838E83E3CFE885F985812FDA
:105F90000995892BA1F3DACFFA01AA27283051F10C
:105FA000203181F1E8946F936E7F6E5F7F4F8F4F4A
:105FB0009F4FAF4FB1E03ED0B4E03CD0670F781FA9
:105FC000891F9A1FA11D680F791F8A1F911DA11D8E
:105FD0006A0F711D811D911DA11D20D009F46894C7
:105FE0003F912AE0269F11243019305D3193DEF66F
:105FF000CF010895462F4770405D4193B3E00FD025
:10600000C9F7F6CF462F4F70405D4A3318F0495D0F
:1060100031FD4052419302D0A9F7EACFB4E0A695F2
:106020009795879577956795BA95C9F70097610514
:10603000710508959B01AC010A2E0694579547956A
:1060400037952795BA95C9F7620F731F841F951F5F
:08605000A01D0895F894FFCF94
:106058000100000000000000000000000000000037
:106068000000000000000000000000000000000028
:106078000000000000000000000000000000000018
:106088000000000000000000000000000000000008
:106098008080800000000000000000000000000078
:1060A80000008080C0C00000000000000000000068
:1060B80000000000000000000000000000000000D8
:1060C80000000000000000000000000000000000C8
:1060D80000000000000000000000000000000000B8
:1060E800000000000080C0E0F0F8FCF8E0000000CC
:1060F8000000000000000000000000000000808098
:106108008080800080800000000080808080800087
:10611800FFFFFF000000008080808000008080007A
:106128000080FFFF80800080800080808080008069
:10613800800000000000808000008C8E84000080B9
:10614800F8F8F880000000000000000000000000DF
:1061580000F0F0F0F0F0F0F0F0F0F0F0F0E0E0C077
:106168008000E0FCFEFFFFFF7FFFFFFFFFFF000056
:10617800000000000000000000000000FEFFC70152
:1061880001010183FFFF00007CFEC70101010183BB
:10619800FFFFFF0038FEC78301010183C7FFFF002F
:1061A8000001FFFF010100FFFF0701010100007F5F
:1061B800FF80000000FFFF7F0000FFFFFF000001DD
:1061C800FFFFFF01000000000000000000000000C9
:1061D80000030F3F7F7FFFFFFFFFFFFFFFE7C7C7FA
:1061E8008F8F9FBFFFFFC3C0F0FFFFFFFFFFFCFCC7
:1061F800FCFCFCFCFCFCF8F8F0F0E0C00001030338
:106208000303030103030000000001030303030168
:10621800010301000000010303030301010303005C
:10622800000003030000000303000000000000005A
:106238000103030303030100000001030100000040
:10624800030301000000000000000000000000003F
:106258000000000080C0E0F0F9FFFFFFFFFF3F1FD4
:106268000F87C7F7FFFF1F1F3DFCF8F8F8F87C7D84
:10627800FFFFFFFFFFFFFFFF7F3F0F0700303000EA
:106288000000000000000000000000000000000006
:106298000000000000FEFEFC0000000000000000FE
:1062A8000000000000000000000000000000E0C046
:1062B8000000000000000000000000303000000076
:1062C80000000000000000000000000000000000C6
:1062D8000000C0FEFFFFFFFFFFFFFFFFFF7F7F3FC4
:1062E8001F0F071F7FFFFFF8F8FFFFFFFFFFFEF8F4
:1062F800E0000000010000000000000000FEFE00B9
:106308000000FCFEFC0C06060EFCF80000F0F81C71
:106318000E0606060CFFFFFF0000FEFE0000000050
:10632800FCFEFC00183C7E66E6CE84000006FFFFFB
:106338000606FCFEFC0C0606060000FEFE0000C079
:10634800F8FC4E4646464E7C7840183C76E6CECC65
:1063580080000000000000000000000000000000B5
:10636800000000000001070F1F1F3F3F3F3F1F0FA6
:10637800030000000000000000000000000F0F00F4
:1063880000000F0F0F000000000F0F000003070EA2
:106398000C18180C060F0F0F0000010F0E0C180C2C
:1063A8000F070100040E0C180C0F070000000F0F58
:1063B80000000F0F0F0000000000000F0F0000008A
:1063C80007070C0C181C0C060600040E0C180C0F02
:1063D80007000000000000000000000000000000AE
:1063E80000000000000000000000000000000000A5
:1063F8000000000000000000000000000000000095
:106408000000000000000000000000000000000084
:106418000000000000000000000000000000000074
:106428000000000000000000000000000000000064
:106438000000000000000000000000000000000054
:106448000000000000000000000000000000000044
:10645800000000AC078000030201002300010013C4
:1064680002000003050400030304100305032000D1
:106478000103070F1F3F7F0080C0E0F0F8FCFE2CEF
:10648800343C444C545C5C00000000E016B31679C0
:106498001882156903A0169116000000000513EE76
:1064A8000B79185F1626108215AB1583159F159367
:1064B80015B2158215CB10CA106C0DC90ECB14AECF
:1064C800143614D7132532642E25303033642E2524
:1064D80030303364002532642E25303033642E2565
:1064E800303264005354455000313030487A00311E
:1064F8004B487A0031306B487A003130306B7A0083
:10650800314D687A0049463A006B004D487A00568A
:10651800464F004C204F0052580038306D00343040
:106528006D0032306D0031306D0033316D00323521
:106538006D0032326D0031396D0031366D00313306
:106548006D0031316D0057464D0041495200545598
:0865580000534D0054580000EF
:00000001FF
